:020000040009F1
:280000000108006999994204204EB1FD0400FFFFFFFF4006000000A0027020020A00280009000000000000001D
:FB002800411A0042726F6164636F6D20426C7565746F6F74682044657669636500980100035C0100017206000300000800017A020000089304002000000068040012000C006A3600030012000000B0000000A0000000431008045310020180000000900000006310040273100402C1000000D000000020000000300000007C04000100000209080068000F00030000006F210002001F05C9000000AA147F8C00FA000040970000000014000002081E000000000069020049045D0C000A64E6B000008898425A33435F09003C280100040004F70C0A6F0098160800C600F3025D0066033000C900E10268005C033600C300E2026A0053033C00C200E1026C0046
:FB0123004E034100C500D60272004A034300C300CE02790042034800C500C00283003A034E00C800BF0282003B034E00C900BC028400370352000808070707070707060606060505050502C0500194FC0E00FFFF00005E02000030FC0E00FFFF0F006304000000FD0E00FFFF0F006602000088FC0E00FFFF0000000200002CFC0E00FFFF00004904000070FC0E00FFFF00000B09000074FC0E00FFFF00002E010000D8FF0E00FFFF000062190000D0FC0E00FFFF000020C90000C8FC0E00FFFF000038850000DCFC0E00FFFF00001CC80000CCFD0E00FFFF0000048000005CFC0E00FFFF00000200000020FC0E00FFFF000019210000E0FC0E00008000000068
:FB021E00000000C0FC0E00FFFF000022000000948F0800FFFFFFFF000F000F988F0800FFFF0000000F00009C8F080000FFFFFF00040404CCFC0E00FFFF00002B45000068000F00FFFF00000308000078000F00FFFFFFFF0504040430010F00FF0000000D0000008C000F0000F0FF0F0000800834010F000F000000080000001C010F000000FFFF000005062C010F00FF00000017000000B0010800FF00000005000000D07B0001040A08FC0E00FFFF00002E3600000CFC0E00FFFF00002CAE000010FC0E00FFFF00002AAC000014FC0E00FFFF0000A222000018FC0E00FFFF00001D2000001CFC0E00FFFF00000D15000020FC0E00FFFF0000858D000024FC53
:FB0319000E00FFFF00008311000028FC0E00FFFF00000001000098FF0E00FFFF00003E410000C3180012691419310870047836042430607180764A3108290B7E07CF090010FF266EF0B009F060D10900010403036B1420206B1A2400FF010808040F000DFC0BF809F407F005EC03E802040F000DFC0BF809F407F005EC03E8020301000182D600040602020A233C5A6E7D80008000800080008000800080028002800280028002800214FF19880AFF610000000000000000000000000014FF19820AFF610000000000000000000000000014FF19000AFF610000000000000000000000000014FF19080AFF610000000000000000000000000014FF190B0AFF3B
:FB041400610000000000000000000000000014FF19100AFF610000000000000000000000000040FFFF68027B0000000040FFFF68027B0000000040FFFF68027B0000000040FFFF68027B0000000040FFFF69027B0000000040FFFF69027B0000000082D600FF0602020A233C5A6E7D80008000800080008000800080028002800280028002800214FF19880AFF200000000000000000000000000014FF19820AFF430000000000000000000000000014FF19000AFF660000000000000000000000000014FF19080AFF660000000000000000000000000014FF190B0AFF430000000000000000000000000014FF19100AFF2000000000000000000000000000FA
:FB050F0041000000007B0000000041000000007B0000000041000000007B0000000041000000007B0000000041000000007B0000000041000000007B000000008612000413004008000040130001000180FF000113C15E0044041422A244041422A23B04B104B204B304B404B504B604B704B804B904BA04BB04BC04BD04BE04BF04C004C104C204C304C404C504C604C704C804C904CA04CB04CC04CD04CE04CF04D004D104D204D304D404D504D604D704D8280C000A0800800208002C012C010B0400184C09000B0400F44C09000B04008A4E090008250000B0DB010078F0A8FC160004650900281CFEF7FDFE281C5F3000210170391C321D87F74DFB0876
:FB060A000F000184E0000030BD00B50000000000000817000288E0000087F0D2F908003054090000F002F800BD0000081D0003C46200008FF0E3FB0E008E5A090001B4FFF769FF01BC70F71FFC000008150004586600008FF016FA0600885A0900FFF796FF30BD0B04002E5C09000B0400585C090008150005C08400008DF08AFE0600D8610900FFF7A6FF30BD082D0006B47702006EF013FD1E00DE61090002B461684907C90F301C91F76BFC02BC002902D0F06991F7E0FA91F7E2FA080F000724B500000FE0C046000000000000080F0008C44F000010E0C046000000000000086700091CF0030057F0EEF85800FC61090070B5061C0C1C151C002B21D123
:FB07050004A8008840281DD105A80088202819D15A2917D8081C15D004F08AFB002811D1032D0FD02204121408210748002304F087FB002806D1221C291C301CA8F7A9FF012000E0002070BD18650800080F000A988000005808042B0000000000000817000B680C040055F0F4FA08005462090000F002F870BD00000819000C64D4000088F078FF0A0058630900281CFEF7ADFF77F796F80813000D08D6000088F0ABFE04006263090077F754F9080F000E80DA0000C046C0460000000000000815000F2452000091F09FF806006663090000F001F8F0BD0B0400C864090008190010845C020070F049FC0A001A6509009B005859EF188FF7B2FB081700118D
:FB08000064F8000086F05EFE08002465090000F002F8F0BD0000081700123CF5000087F05EF80800FC65090000F002F830BD0000082F0013C4F6010076F0D8FF200078660900054B30B4054CE57949190C06211630BC195489F71DF8C046903408008C03080008170014487C02006EF026FD08009866090000F002F870BD0000082B0015D4BA00008AF01CFE1C00106709000AB4201C311C00F009F80ABC012803D0042B01D175F7D8F975F7D9F9081F00162CF0000087F08BFB10004667090001B483F7B5FB01BC00F024F878F76DFC08250017E4A203005CF037FA160056670900002806D100F007F8002802D10120A3F7EAFDA3F7C0FD08170018C06A02D5
:FB08FB00006FF074FE0800AC67090000F002F830BD000008230019C47202006FF012FB1400EC68090008B4301C0122012300F004F808BC90F7E7FC0000920600A300800014190817001A2848020072F024F90800746A090000F069FA8DF733FF0817001BB473020070F084FD0800C07E0900FFF75DFE8FF707FB080F001C34C40100C046201C0000000000000817001D2447020072F0AAF908007C6A090000F0F7F98DF765FE0817001E6847020072F08CF90800846A090000F009FA8DF77DFE0817001F0C4D020071F0BEFE08008C6A090000F099FA8EF754F908170020404D020071F0A8FE0800946A090000F0AFFA8EF76EF9081700217C4D020071F08EE9
:FB09F600FE08009C6A090000F007FC8EF782F9081700227854020072F012FD0800A07E0900FFF758FD8DF7F9FA081700230C57020072F0CCFB0800A87E0900FFF7B4FD8DF77CFC081900244472010081F02DF80A00A2820900FFF7F5FF7EF7D0FF0000081700254C58020072F030FB0800B07E0900FFF724FF8DF7E3FD081700265C46020073F034FC0800C87E0900FEF774FE8CF7D5FB081700270865010080F0CCFA0800A46A090000F0FDFD7FF748FD0817002834AE01007DF000FB08003884090002B0FFF757FF70BD08170029086E000094F06AFF0800E0BC0900FFF78EFF6BF7CCF8087F012AA444000094F0D4F870015086090000B528490B682649B1
:FB0AF1000B6024490B6822490B601E490B682D490B60434B43490B6034490B680120C00303430B6040490B78002B04D02F490B68400303430B602D4A13685B085B0013603A4B3B4A1360B0F75CFEB1F785FAB1F7D4FDB1F77AFF0D21364802F069F9364A9068002803D098F785FFB0F721FD2448244A11684160244A60E0C046C0B00800FFF2011A00AC0900848FB002D08B0E00A0800E0004AC0900148B0E0008AC09006CE505000CAC09008C150800378509006785090041860900BD850900298609005C000F0094830E00FF00FFFF608B0E0040230001E08A0E00E02C0800A4860E0088B2080005000080850000801C800E0014800E00848F080004830E6A
:FB0BEC0000108B0E00C8FC0E00C42C0800CC2C0800D02C0800C82C0800D42C0800D4FF0E00BC8B0E00AD020000CC8B0E001CCD080010325476D48B0E00009D0800ECCC080011684161054A11688160054A13680360044A1368044A136000BDC046D02C0800C82C0800D42C0800D4FF0E000861002B0044000094F01EF852004084090010B5A448002383700423437001230370A14BA2480360A24BA24C2360A24C2368A24C2360A24C2368A24C23602C22A249A248BCF787FAA148A14C2060A149C160A1494162A1490161A14B8361A14BC36110BD080F002CD0B80400A5F809E00000000000000817002D20BA04004DF086F90800308D0900FFF7D4FF30BD22
:FB0CE70000000817002E3069040052F00AFB0800488F0900FFF7C4FFADF70EFD0819002F545D040053F0FCF80A00508F0900B3F786FFFFF7B2FF30BD08190030E0A504004EF0BBFC0A005A8F090000F003F803B0F0BD000008170031E882040050F08AFE08000090090000F002F830BD000008170032B0B104004DF0A4FF0800FC90090000F002F830BD0000082B0033DCC004004DF070F81C00C0910900FF233D3343430448C0189F300078002800D101207047C046349D0800081B003494AC04004EF0ACFA0C00F0910900201C00F003F8B1F750FD0000081B0035ACAC04004EF0ECFA0C0088920900201C00F003F8B1F710FD0000082300363CC104004D6B
:FB0DE200F04EF81400DC91090029187F231B02FF339D4200D35D1EFF23B2F7A8FF08170037981B030067F0EEFB080078930900FFF7D2FF30BD0000082B00381C7B040051F048FC1C00B093090004910FB4301CFFF7E3FF012802D10FBC05B0F0BD0FBC062DAEF7AAFB081F003918AC04004EF014FC10004494090003D1FFF7C1FFB1F7E8FBB1F7E7FB0000080F003A1C730400C046C0460000000000000817003B807A040051F0A0FD0800C49509000420AEF766FE10BD0817003C9882040051F098F90800CC950900FFF7CAFF30BD00000817003D6CA804004EF066FF08003C970900FFF74AFFF0BD00000815003E94A304004FF072FB06007C9A0900FFF74C
:FB0EDD00E8FF10BD080F003F0CA3040000F01DF8000000000000082300404894000090F01BFB1400829A0900012B02D10020287001E06FF7E8FC62686FF724FD081D0041A4CC04004CF0F7FE0E00969A09002878B2F785F8201C00F001F830BD080F0042C4A904005E4A2068000000000000080F0043A4630400FE23F533000000000000081F0044D472000092F0F0FB1000B89A0900301C049900F004F8009988426DF708FC081700459897040050F0BCF90800149B0900FFF79FFEF0BD000008170046E49D040050F088F80800F89E090000F002F8F0BD000008150047D099010080F0DCFB06008CA10900FFF7B2FF00BD0815004868E901007BF013FC06B4
:FB0FD8000092A10900FFF7C2FF00BD08230049A4E901007BF0F8FB140098A109000FB4301CFFF7C6FF0FBC0A22311C84F7FFFB00000817004A70EF00008BF058F9080024A20900FFF7C2FF74F7A8FE081D004B645F040054F062F90E002CA20900607D01386075FFF7C7FFABF798FE0819004C14FF00008AF091F90A003AA20900FFF7E2FF75F76EFE00000877004D7461030064F066F8680044A2090010B500248BF73AFF012803D309D0022820D102E09EF784FB01E0A3F7ECFE041C18E00D490B78002B14D00C4A106803680B4A13600B4A1378002B0BD08B784978002B03D04B00FF21013101E04B00802199400160201C10BD481B0800E40A0800AC58EC
:FB10D30008003A010800080F004E7C640200131C03600000000000000857004FB462020073F0FAFF4800ACA2090000B50D490868002804D003280FD0052811D104E009480378002B0CD007E0084B18680122002199F756FA9BF728FE05490B680120186000BDB0C80800D1CA0800F40A0800E40A0800081B0050C0B903005EF098FC0C00F4A20900211C00F00BF8061CA1F764FB081F0051B49D030060F0A4FA100000A3090002B400F015F802BC0C68E3069FF754FD081900527847000095F074FF0A0064A60900381CFAF723FC6AF788F808190053AC47000095F05FFF0A006EA60900281CFAF73CFC6AF7A1F8081B00543CDB00008CF09CFD0C0078A60900
:FB11CE000081B000F003F873F7C2FA000008270055405B010084F010FC180064A30900002E02D00020E05504E0E35D002B01D0013BE3557BF7FBFB081B005650A704004EF0FEFE0C0050950900381CFFF7F4F902B0B1F7FCF80817005758A704004EF000FF08005C950900FFF712FAB1F709F908210058B03C010086F05EFD120070A7090001B4301C00F010F801BC74F7A3FC79F799FA081D00595CB503005FF011F90E0082A7090001B400F00FF820BC6B01A0F7E8FE0817005AA8A0030060F072FB080090A7090000F015F89FF7A4FC082B005BCCB203005FF08EFA1C00ECA709001378002B07D103B400F008F8012803BC01D1A0F768FDA0F772FD0000DF
:C512C900081B005C74B403005FF0D4F90C0020A8090000232B7500F02CF8A0F726FE081D005D1C69020073F086FF0E002CA8090003D100F027F8A1F7D9FF8CF774F80827005E30BB03005EF083FE18003AA80900012D03D1002E01D100F05BF8A068A1F7F4FE0021A1F772F90827005F0862020074F023FB180052A80900201C08B4019900F01BF808BC9C4201D08BF7D3FC8BF7DDFC082500609CBC03005EF0E5FD16006AA809001B0705D400F049F8002801D1A1F713FAA1F73EFA00000A05002DCB080001FE000088
:FB4B0000F0B54A4C4A4B4B4803604B4B4B48036001F07EFF00F0ECFB00F0FCF900F0ACFB00234748037000F007FB00F019FB03F0F6FE444A151CE435434B2B60434E336802263343414E33604148036880218B43036000233F4E33703F490B1C23333F4E33603F4B3F4E33603F4B404E33600B1C12333F4E33603F4B3F4E33603F48404B404E3360031C0E333F4E336012233F4E33700B1C11333E4E33603E4B3E4E33603E4B3F4E33603F4E31603F4B3F4E33603F4E33683F4E33603F4B404E3360404B6B67404B061C071DC8C40E363E4FC8C4991C0E30061CC2C43C4BD36200233C4E336004F025FF3B4B6B65E4209EF73AFB0007000F042805D13F20C030
:FB4BFB0043364A5073000A9073002335490B703548E86235490B70F0BC08BC184700B533483349086033480849C86400F03BF900BDB8AA090039530900BCC808003D530900F0C408002DAE0900A0190800595409006C010F0040150800FD0708001E45000014AB090020C9000018AB09001CC800001CAB090020AB09003885000024AB09005E04000044050000881308008C13080090130800781308000EC90000801308000AC800007C130800841308002685000074130800D8FF0E0028AB0900621600002CAB09000D5A090042050000621900005594090010AB090061660900B813080078AC090041A0090079AC0900014B0900900008008D64090070B59A
:FB4CF60000200F49104B4B6114E06B099C00EB06DB0E01259D400B592B430B5143004C69C50052195268012632432725AD03AA1A1A530130054AC3009D58922DE5D370BDC0464C1B080068AC0900A8A909000020704700207047002801D0002000E0012070470020704710B5037814490B700620A9F757FD041E10D00E230370042343700023437101238370F723C370FC230371A9F771FD201CA9F748FD012010BC08BC18478105890D030AFC201840FC2803D1F72901D1034800E000207047C04678AC09005D4D090004280AD106480378002B06D0054803785B065B0E0370012000E000207047C04678AC090039C3080030B582781202437813439A059224
:FB4DF1000D1B0AFC252B400C2B05D1032A40D105F0F1FA01203DE00124FC2B32D1B52A15D0B62A16D0C22A17D0C32A18D0C62A2CD318D0C82A19D31BD0CB2A1CD9E62A02D0F52A22D11AE003F0C2FC1FE001F0D5FEDFE701F008FFDCE701F037FFD9E701F07DFFD6E705F0FCFAD3E705F036FBD0E705F073FBCDE796F7E2FCCAE703F01DFAC7E7202B04D0042B02D10024201C00E0002030BC08BC18470248024908607047C046E54D090018C908000020704701480249886070479D4E0900201A080030B5051C7AF706F9041C281C8AF795F98749201C2830062205F026FD00280BD1844C2560012363717F21C943A01D072205F022FD00232371002030BD3E
:FB4EEC0010B5041C0120A040C1437C4803680B40036089F7C9F878480368A34203D1FF2303600023437110BD75487649C8607047F0B583B0041C012906D164300023C372251C9435AB73EB736F4803689B079B0F032B02D071F7D4F9C8E00023A381E07B484000D1B6E070F76FFC002803D1674803691B0101D5012100E00021271C64373E1CFB6880208343C8010343F3600C365F4A1078431006D0C3071B0E31688020814319433160594803691B0102D4381C94F74CF9BB69002B02D03B681B063BD4338868460380E37B012B0DD0251C94356B7B002B10D02B88042B0DD3EB7C022B0AD3AB7D002B07D1A72303201855009B78208343002106E00121E912
:FB4FE70074009B78208343082003431F20800283438802034300931B041B0C3F4A1360012030723B4A13691B0152D400984006010F00231A1C012094F72CFB45E0E07B002802D1A72301221A55012804D1E37C042B01D072F71FFCF37A002B06D00023F372336801204002434033600121B172251C9435A97326480369DB0002D5201C87F72FFD338824490B60B0884860381C70F74FFC30684006030F2048C05C3072431EA381E37B002B0FD10121387F81401C4A1068084008D1E37C042B05D019480378AB7519480378EB75114803691B010FD5201C94F785FE0BE0271C64373B727B7270F7DDFB636C002B02D05A231B5BA38103B0F0BC08BC184709C178
:FB50E200080030AB0900000408001D4F090000020800188B0E0054200800DCC80800CC8A0E009EBB0500B4010800F5010800F601080030B50D1C041C75F723FE6B075B0F012B05D1E37B002B02D1A07B9CF762FD30BC08BC184700B52C2204490548BFF720FC034804494161044B186000BD0CBD050040AB090015510900E402080010B53F4C3F4B1C602C223F49201CBFF709FC3E48606210BDF0B5041C051C876A28353B4B42331878002866D1201C012172F77DF9061E4BDD022804DB201C77F7F7F9002859D1618C8B1F9E4223DA304A13689C420BD0391CAB310878013800D30870731C5910201C76F784FF30E0731C5810E37B002B05D07B6C002B02E2
:FB51DD00D06B7F002B25D02F89B84222D36A89002A06D1A389002B03D1201C71F78BFD18E0BA4200DA3A1C904201D90C2310E04B23A27C1B5D9A420CD102280AD36B7F002B05D014480378994201D9282300E03823A374211C4D31087800280FD00238087000060BD1E37B012B02D0237D0C2B05D0321C201C0523022177F7E0F8F0BC08BC18476CAB09000003080074BD0500795109006C210800F402080000B52C2216491748BFF780FB1548164B18601649016100BD30B50D1C041C77F7C8FF022D09D16B23185D002805D0201C87F7B1FA201C87F7E9FA30BC08BC184700B5011C6831CB78002B07D04B7A002B04D18B78002B01D087F7C0FA00BDC04624
:FB52D8002CBE050098AB0900300308009152090000B57CF7FEF900BD00B52C220B490C48BFF744FB0A4B0B48036000BD0A49CB6ADB0007D5094AD3885B00418C8B4201DC012100E000215A3001707047B0CB0500C4AB0900F403080054200800942008000020704730B5041C002957D0012946D140051BD421E02D4D291C2D48B7F773FF2988281C262902D103F0E1FD0EE0042902D17CF7BEF909E00F2902D104F0D2FB04E08900234A8958C6F799FA2048B7F772FF0028DFD0204B1C4020042ED51F49086803791E490B7000230371B2F7E7FE79F774FE002803D11A48437D002B09D019487AF7A6FE80F7EFFF1321162004F009FF01E07AF75DFE144B1CA8
:5D53D300400EE002290CD1C00308D50E490878012804D10B490B681871B2F7B8FE7BF74BFF201C30BC08BC18470A480B4908607047F4440800284508009CBE0500FFFBFFFFC04F080079AC0900E44E08001C450800FF7FFFFF3D530900F0C4080092
:FB54380000B5431E04490B6004490B78032B01D1BFF75EFF00BDC046E08A0E0038080800F0B587B0061C0491081C00210391A34C2064211C4431009100238B70A0488568002D00D16EE2AB7D002B09D0012203920023AB756361237810208343237006E06069002803D0012E01D970F777FE22691D27FF03002A50D0607A012803D19389002B4AD047E08F4B1B5C002B43D1BB68DB0742D4137D092B3DD204281AD1012E18D196756261237810200343237023683B6085490B687233187802282DD0002382490B608249086882490B6803600B68036022E002280AD1012E08D196756261237810200343237023683B6015E0032803D179498B78022B0FD0066B
:FB5533002801D0032805D1012E03D1BB689B0600D5C0E1122803D0102801D070F7A1FD6A4B985D029000287DD00123DB07334301936B4B6C490868986301236B490B606B490B689B0C9B040B600B6869490868034366490B6001230099CB7066490B6866490B6066490B6866490B60287C1A281DD164490B6864490B6064490B6864490B6064490B6864490B6064490B6864490B6064490B6864490B6064490B6850490B60634908686349086063492DE063490B6855490B6062490B6855490B6061490B6855490B6060490B6855490B605F490B6855490B6019280ED1FF2017302B562A3309DD5B490B683E490B605A49086851490860594908E059490B6856
:FB562E0039490B60584908684C4908605749086857490860A87B2318042801D3187800E0205C6F2290431870C2E0A87B225C0F218A433107090F0A43225423180428049802D38107101C01E081071878490E6022904308431870234B464908689863009AD378002B00D1A1E022490B689B0C9B040B600B684049086803431D490B600023D3703D490B681D490B603C490B681D490B603B490B681D490B603A490B6821490B6039490B681B490B6038490B681B490B6037490B681D490B6036490B6809490B6035496BE0642C08006C210800ECBB0500DC02080060000F00AC2C080044020800882B08002CFC0E0060020800E08A0E00B88A0E005C0208006C65
:FB572900130800D8FC0E0070130800E0FC0E0014AB0900CCFC0E001CAB0900DCFC0E0018AB0900D0FC0E0024AB0900C8FC0E0020AB0900D4FF0E00D0AA0900D4AA090030FC0E00D8AA0900781308007C130800801308007413080084130800B8AA0900BCAA0900C0AA0900C4AA0900C8AA0900CCAA0900D8FF0E00B82C080048020800BC2C0800C02C0800C42C0800C82C0800CC2C0800D02C0800D42C0800D82C0800DC2C080008689349086093490B6893490B60002101912868826A281C0021C6F763F8002810D026231A5C002A0CD08368002B09D00298002804D0802301981843019001E0012200E00022237880208343D00103432370202004990840D1
:FB58240001D00120C0037F4908600499090704D47D490B68802083430B600499880801214140A27880208243C8010243A2702868826A281C0321C6F729F874490B78012B01D076F7C9FF05A9714A13687020034018099CF716F82369002B14D0637A032B11D188F777FB002806D16A480368032B02D00368062B06D12B7C122B03D101230098837058E005988007800F06D003280ED1069B60490888834209D30398012800D1656170F7E4FB012300994B7043E00820B860A87B786223683B603B1C1833221D03929207920F02D1039909680FE00399891A0391D2000968D140049120218A1A03994968914001B40598014301BC1960BA69331C103B042B0DA2
:FB591F00D2474B1340FF22013282401343BB61102E07D1444908684449086002E040481040B8610198002800D07861E5602672002300990B704B70281C8CF72BFC012007B0F0BC08BC1847394B3949087A185C39490B68002814D00120800303430B60364A136836480340364A117849020B43354A1360354A1368302083431020184308E0324803400B602C490B682E490B602E4908682F490860704710B5254C234B607A185C002802D070F7D5FE15E06069002801D070F7DFFB27490868637A012B01D1254A00E0254A13680360116801600023234A136070F7EAFD002322490B60E3602361637244340120207010BD002803D10348036803480360002065
:6E5A1A00704730FC0E0028AB0900D8FF0E00648B0E00A4860E00D4C1080024860E001C840E00E4B60800FFF0FFFF9406080064FC0E00ECBB0500642C0800808B0E00B02C0800FFC1FFFF9013080088FC0E00B42C0800FFBFFFFFCCFD0E00AC2C0800400208004402080060000F0018800E0051
:FB5A9C0070B582B0061C65480168890602D5022072F795FB624C2568A3682360002D26D0002E18D19EF76AF9002814D0C30703D52A68916900290BD1430703D52A68D169002905D1830706D52A68116A002902D0281CC5F7E2FE9EF76EF9011C2A685269002A04D0002802D0281CC5F7D3FEA0680026A84218D0002D21D02A681269002A03D0281C0521C5F7C5FEAE8123699D4200D126612B7D092B11D3281C73F75EFD281C73F7E3F80AE0002808D06369984205D166613B4800220121B7F793FE3A48C16E002904D0A368002B01D1C5F7A5FE70F72CFBA06800284BD08681037D092B20D26369984205D166612E4800220121B7F778FEA068A84206D1014E
:FB5B9700684968002902D00523037508E0017D032901D0042905D101684968002901D0C5F77EFEA0680223037501680A69002A02D00221C5F771FEA068807B1D4A136870210B401909884216D169469BF760FE70F7D6FB002801D0174800E01748028800998907890F04D0032905D1019B934202D33F2301201855A0688CF756F901208CF766F9A66066603C3426716671012002B070BC08BC18470948044988617047C046C4C408006C2108000C2D0800201A080024860E0066020800640208009D5A09009F48A0498865704700B59F4A9007800F01D1116808E0121AC0001368C3402021081A516881401943C90F98480170984A1068002817D0974A02607B
:FB5C9200974A8260974AC2600123964A13700023964A1360964A1360964A1360012902D100F007F802E04068C5F7FBFD08BC1847000000B500F003F808BC1847000010B564238C48037000238C4803608C4803608C4C236000F04FF87D4A9007800F01D1116808E0121AC0001368C3402021081A51688140194301204007014015D081490B68001403430B6080490B68804803400B6004390B680120800303430B607C4B7D490B6003037C490B60684A9007800F01D1116808E0121AC0001368C3402021081A516881401943C90011D5744C2368002B02D0201CB7F77BFB7149201C00231A1CB7F756FB6F480168201CB7F75CFB8EF7D8F910BD10B56C4C2339
:FB5D8D0068012423436A4C236001239B03694C2360504A9007800F01D1116808E0121AC0001368C3402021081A516881401943090105D55E480368022003435C4803605D4800218160F421C16020210161E8218161E9214161102141624021C161016205239B04036010BDF0B582B0071C01910C1C0022009201235B0250490B604E490E68360C3604211C242903D0151C25291CD102E008240A210AE070300078022802D10824464801E0012446480278012123010D031D4313071B0D1E43FB7B002B00D1E4E00123DB031E43E0E0019B5B003D481C5A3D498C4211D18023DA5D3C48135C1B013B4818188388002B07D0374C1034837A012B06D1344C2034D6
:FB5E880003E0002C01D1251CC3E0381C8CF712FB002800D0402431480368002B07D0602C01D1E02464E0702C08D1D02460E00198042801D0022801D101252D04302C4FD17023D85D00284BD0214C703450E0C046615C0900A0190800C005080030C8080044060800C55C0900F55D090029600900B805080034C8080038C808003CC80800D005080040C8080048C808004CC808009C800E0010800E00FFBFFFFFFF030000BC820E0010000C0068500800673D0200D405080070010F005C000F0074820E000C800E009806080090060800D8050800100100009005080024500800D4C40800502C05D13B6FDB0502D501235B041D432543FF23113370339C4203DA
:FB5F8300D023095D48C15C0091302C0BD17023D85D002807D1381C2830037D807A19180906090E0091009803031D43FB7B002B02D00123DB031E43FB7C032B04D1788CC306180F03021E43402C25D14C480378002B06D0381C8DF7EAFD03071B0A1D431AE00123DB041D43B87B9BF775FC4008444A1060444A11689BF709FC434A1060434A1368984204D2381C8DF7B0FD002802D001233A4803703E480560466002B0F0BC08BC1847F0B582B00F1C051C0022009201908CF741FA364E002844D034682F48017800291AD1A87B9BF745FC40082C4A10602C4A11689BF7D9FB2B4A10602B4A1368984204D2281C8DF780FD00281BD0012322480370274B1C40DD
:FB607E0015E06B6E1B0612D4012910D1281C8DF770FD00280BD1A87B9BF720FC41081A4A11600023174A13700123DB041C4314480378002B03D001988CF7AAFE0090174B1C40009803071B0A1C433460042F01D0022F05D13368012109040B43012107E010480378002B06D033680E490B40002133600B48017002B0F0BC08BC184724060800B805080038C8080034C808003CC80800CC05080070820E00FFFFF7FFFFFF0FFF45C80800FFFFFEFF30B5041CC37C032B27D1037D0C2B24D11830437B002B20D121490B699C4202D18B68002B13D0418900680B1858010509A07B9BF7BEFB854201D3281A03E0431B01200007C01A831F1648834205D3201C7391
:5F617900F73EFA201C72F7CCFE237D022B03D0032B01D0042B07D10F480379002B16D0201C70F715FD12E00C480369002B02D0201C6FF7AAFF06494123585C012804D0002804D10B689C4201D172F738FA30BD6C210800FBFFFF07A42C0800642C0800DF
:FB625C0070B5041C00253848436912219B0708D5364A1068364A106050304079122800D8011C43209CF7E2FF324BA360324B2361201C0830AAF783FE2168086063681D60AAF7ECFE201C1030AAF779FE216808600420AAF7FBFE6061062801DAAAF7DEFE201C0830AAF76BFE216808606368002018600420AAF7EAFEE060201C1030AAF75EFE216808606368002018600420AAF7DDFE6061E368C61A301CAAF72DFF042817DD01350C2D14D0301C042E08DDAAF723FF8100081A2169081802382061CFE7AAF71AFF8100081AA168081A0230A060C6E7A16820690B1AE3614018C30F18184310236270BDC046181B0800D4CC0800F4AD0900FF03000001FCFF99
:01635700FF46
:FB636C00F0B5444D2B68987B9BF7B1FA46082B68996C301C9BF746FA041C2868011C94314A88002A10D094420ED9037D0B2B0BD00D2B09D070F715FB2B686433197F012000037AF7E7FF64E00B7D002B06D0CB88F31A1B041B0C9C4200D81C1CC36F6430002B06D00B89F31A1B041B0C9C4200D81C1C8A88B31A1A04120C944200D8141C0B881F1FBA4204D3CB7C022B01D30023CB74214E33889C4204D80020BA422ED303202CE073889C4201D8042228E0B3889C420BD9007F74F737FE002814D0037C112B11D115494B889C4203D829689431052215E08B889C420DD82968943106224A745E2383740CE0F3889C4203D829689431062204E02968943107BA
:9D6467002200E0021C4A740B7E012B04D1531F012B01D804234B74F0BDB421080034020800EC02080010B5A3F749FB0B494B699B070FD50A48036801200343084803600A249BF7C6FC013CFBD1044803685B085B00036010BC08BC1847181B0800F0FC0E0010B5094C2C220949201CBEF757FA0849E160084B1C6010BDC27B4A4002D0838C05490B607047C046F8AD090034CC0500E164090010040800CC8A0E00BD
:D0652C00F0B581B0041C00210091C56D8726F600002D04D1301C9BF71CF8051E03D0301C9BF717F80090264F3B68002B08D1301C08309BF70EF83860311C0831BEF72EFD20480368002B0DD1301C08309BF701F81C4A1060311C0831BEF720FD19480368002B07D03B68002B04D0002D02D00098002817D1E02300201851E565E4210B59DB0208D46358104803430B515022206807217DF74CFA0D480368002B0DD19AF7E4FF0AE0E5656060E4221359064883431351206807217DF75BFA002001B0F0BD444408009C4408000000100060030800C7
:7466040030B5E4221358012109058B431350051C79F7A0F90024002800D0EC65E86D002802D09AF7D1FFEC656868002802D09AF7CBFF6C60074D2868002802D09AF7C4FF2C60054D2868002802D09AF7BDFF2C6030BDC046444408009C44080000231360012805D10123DB040B6007239B031360704700000F
:7066A000B0B503685B011948C21880270F404906490E9068002827D00568281C041C002F06D0437B8B4201D0002300E0012306E0037B5B088B4201D0002300E00123002B0FD0A84205D1137C002B02D1D37F022B0AD0111C08319BF732FD201C9AF720FF02E00068A842D9D1B0BDC0467C290800CA
:1A672C0010B5002907D0041C70F70EF9201C6EF779F8012000E0081C10BDFC
:40676C0000B50D48B6F77DFD00BD30B5051C00240A49A300C818C378AB4204D1A300C8180421BEF71BFC0134082CF1D330BD00B50068FFF7EAFF00BDB8520800504708000A
:FB67B40030B5104D0D24281C0022111C90F796F9281C90F789F92035013CF4D130236343094818182C23195C022904D1406A002801D09AF7F1FE0134022CEFD390F73EF930BDC0467C29080080590800F0B582B0051C0E1C041CB0346946207B9BF749F82C482D4A1178431AF6000198991940182A4B984201D3032005E00121284B984200D30221081C009943185808031D5808860176092188301C9AF7E0FF6788391C77F75CFA381A4308AB80831958014009A0601422291C1B4804F074F802B0F0BD10B5041C184908680007000F01280BD80B683F2000020340190A144A906EFFF7B5FF134A9378A37410BC08BC184710B5041CB3F72DF80F498B780085
:3D68AF002B07D1A37C0B498878834202D0201CB3F7FDFD10BC08BC18470E020000DCAA0900A90300007102000000980E00A88B0E0038B0080074150800AC210800D5
:FB690000F0B584B0061C181C01AB07C300252C1C04F02AF800902F1C0199002918D0F37F022B15D1337C351C002B01D00C3500E008352A68101E00D01068002A07D01168914201D12C6001E00B6813600C6014E0357412E00A6801928A4201D1F76001E013680B6001990F60002C04D0236813602260141C01E0141C1260F1680029E9D115E01A680193111C9A4201D1B76004E0136801B40298036001BC0F60002C04D0236813602260141C01E0141C1260B368002BE6D1002D0BD02A68002A05D0136803602B681860286007E02860006004E0F37F022B01D10323F377009803F0CCFF12E02068051CA04201D1002401E0036823602F600399002904D00277
:7969FB009900229CF7A7FD01E09AF79CFD002CEAD104B0F0BD0A480B4908600B480B4908600B480C4908600C4B0C490B600C4B0D490B600D4B0D490B600D4B0E490B607047DD71090064C808003770090068C80800FD76090080C808002D6B090054C808001D6E090070C808007D77090078C8080008AA0900B006080002
:FB6AAC0070B5051C7BF7CBFF011C041CEA691204D20F2273032363730C34414B186800090226800706D5F42043599B0702D5A6703C480660F4204359DB0601D4002A01D1002000E038484860281C90F75CFC0023364A137070BD30B5041C0D1C7BF79FFF33494B681A7BD207D20F0273052343738573304A4260011C201C90F744FC30BD10B5041C0321FFF7E6FF294A5368987B244A1060201C8DF746FF10BC08BC184770B5041C7BF77BFF011CE2691204D20F027304234373F8231D59837B0126B34335402B438373F8263559AD07ED0F0226B3436D002B4383730C30002A0CD1164A537815785B199578EB18D578EB181579EB185279D31800E00023C398
:FB6BA700700F484860201C90F700FC70BD00B5094A5168897B8B07DA0FC907C90F8DF742FF00BDC046641B080088500800D34902005CC80800F44408009F720900E8500800094A020010B5041C6D4A1068C00702D4112323702BE008790002C9780843012177F7E5FF002803D0F8221158490701D51223EEE7C169090403D4F4210B589B060DD55F4B19684906490FF42212589207920F914203D15B490B78002B01D00C23D7E701230B7028342370FFF72BFF10BD30B5051C0C1C031C28330120187001F0F4FA002801D10C2022E020790002E1780843012177F7ABFF00280BD0F8221158490701D40B2013E0F43003685B0601D40E200DE042490868400652
:FB6CA200400F022808D1414A1188601D01F040FA002801D10D20287030BD30B58A7B002A01D1122340E0374CCB7820680225002B06D0012318432060364803682B4305E001239843206032480368AB43036031480B7903704B7943708B7983702F48CB79202B02D12E4B186002E02D48402BF9D0487A00020B7A184340102A4B1860C0006080C87A00028B7A1843204B1880487B00020B7B1843244B188024480280CB7B244803700B7C2348037030BD164A1168C907C90F817317490B78C3734B7803748B784374164A1168090A8174164A11684900C174090A01750D4A11884175090A8175114A1188C175090A017610490B8843760F490B7883760F490B9D
:FB6D9D0078C3760E23C3707047C046641B08005CC8080004AB0900301B0800A80608001E200000940608003A4000009006080006AB090008AB090025AE090026AE090010B5041CFF20052193F7EFFE002806D016238370C470210A017193F771FE10BD10B5041CFF20052193F7DFFE002806D018238370C470210A017193F761FE10BD10B50024201C00F0F0FB0134042CF9D31821AB48BEF7CAF801F04CF8A9480268D10708D55106490F022904D1A64A116872230B4313600023A4490B70A4490B704088C010A3490860A3490B7010BC08BC184730B5051C00244E2363439F481818811C281C062203F049FD002803D1201C00F0BBFB02E00134042CEDD3AD
:FB6E980030BD00B500214E204843954A8218507800021278104302D08DF74EFC07E001310429F0D300238F490B708DF77EFD00BDF0B5061C04250024894F4E206043C019811C301C2830062203F01AFD002801D1251C02E00134042CEED3042D0DD100244E206043C119487800020978084301D1251C02E00134042CF2D3042D18D24E236B43DC19311C2831A01C0622BDF72EFD5C20805B2070000A6070311C201C083000F0F6F9311C28316F480622BDF71EFDF0BDF0B5041C0F1C00264E207043684BC518A91C381C062203F0DAFC002803D00136042EF1D326E0201C78F7F4F9291C0831201C00F085FAE0690F21C9050843E061201C0F23038630308687
:FB6F93008D69780C022A781443A64205D0584A0121B14013688B431360554A0123A3401168194311608485012000E00020F0BD10B582B006224F496846BDF7DAFC002469460623634340481818062203F09BFC002801D0012003E00134042CF0D3002002B010BDF0B582B0071C062243496846BDF7BFFC0024344E0622151C65436946A81903F080FC002806D1391CA8190622BDF7AFFC012003E00134042CEBD3002002B0F0BDF0B5041C0E1C171C344DFF2001302058002801D0B6F70AFAF8210859C00700D491E0002E00D18EE0002F00D1A5E00859800700D4A1E0201C6DF739FCE069F821884340210843E061F822105904229043F8221051201C90F7D8
:FB708E00F3FC206800216DF761FC164A1378002B0AD0E06900043CD41B4880791B4A1178014001D1002832D1261C5C36318800231A1C181C94F718F83088FFF798FE00232B70084803701048037022E0C0467AAC0900641B0800301B08005CC808005DC808009006080025AE090092AC0900BFC10800B7C10800D0200800F8A9090000AA090024AE0900F0AB090026AE090001232B70201C28308DF7FDFAE069000414D48DF71AFB8DF7EAFD012801D18DF709FB98210859C00008D5E06C032189068843E064201C012180F7F5FF0023B9490B70A36B1B072FD5E06900042CD4B6494B681B0528D5201C01218DF7AFFD23E0B2490868800715D5F822105908B0
:FB71890021084310518021E069000400D44900AC4A11600120000778F78CFD002E0DD1201C8DF738FC09E0E069000403D5201C8DF7E4FC02E00123A34803700120F0BC08BC184700B5FC300068002801D0B6F744F900BD70B59D4D03685B019C49CE18041CFFF76DFEE069000403D4201C00218DF76EFD20687CF725FC201CFFF7E2FFE0690006C00E0A2817D1012120688140904803688B430360201C74F737FCE069F821884340210843E061206883F75AFF201CA030042103F0A3FB211C301C01228FF752FCE069F821884318210843E061F82108590721084340218843F8210851206801218140CA437B490B6813400B606DF784FAE069000402D42B78C7
:FB728400012B04D05C342088FFF7A6FD01E000232B70012070BC08BC184700B5011C1D2078F77EFD08BC18470000F0B5071C00246B4E0622151C6543391CA81903F02AFB002805D1A8190621BDF77CFE012003E00134042CECD30020F0BD70B5061C00254E236B435F481C18A11C301C062203F011FB002803D00135042DF1D310E0221C25329107890F01D1106808E0521AC9001368CB402020411A50688840184300E0002070BDF0B5002900D1ABE0041C00D1A8E0C8694005400F2070C8698004400F6070486BA21C93079B0F01D1106006E01070000A5070000A9070000AD070886BA21D93079B0F01D1106006E01070000A5070000A9070000AD070C86A
:FB737F006B221C0A3293079B0F01D1106006E01070000A5070000A9070000AD070086C221C0E3293079B0F01D1106006E01070000A5070000A9070000AD0700D1C50352888A074000AE074AB782375EB786375CB7BA3758B7EE375CB7E237624480378637698204058400FA076E889E076000A20770F1C9C37B86D221C1D3293079B0F01D1106006E01070000A5070000A9070000AD070261C2036C86C4001C00F7070C86C0001C00FB070C86CC000C00FF070C86C8000C00F30711022291C1031701D17E05CC80800181B0800641B0800D45008005DC8080024AE09007C290800E4C70800B4C408007AAC090092AC0900E0AA0900BDF788FA1022291C2031BE
:FB747A00301C1530BDF781FA4534F8782070F0BDF0B5002800D1B8E00C1C00D1B5E04978CB0022785207520F1343C2693F2109028A439906890C0A43C261A31C9A07920F01D1196808E09B1AD2001D68D54020218A1A5968914029434163A31D9A07920F01D1196808E09B1AD2001D68D54020218A1A5968914029438163231C0A339A07920F01D1196808E09B1AD2001D68D54020218A1A596891402943C163231C0E339A07920F01D1196808E09B1AD2001D68D54020218A1A5968914029430164061C5036E17C0902A27C11433180637DF370237DB370A37DC373E37D8376237EC376A37E98210A58D200D208191C1D2349070A4398210A50217F0902E244
:FB7575007E1143F181071C9C37221C1D329107890F01D1156808E0521AC9001368CB402025691A55688D401D43BD65251C20356B78002B04D0C16C012292061143C164AB78002B04D0C16C0122D2061143C164EB78002B04D0C16C012212071143C1642B79002B04D0C16C012252071143C1641022691D301C1030BDF7CAF91022291C1531301C2030BDF7C3F945342078F870F0BD10B5042810D24E21414334484418002020706070A01C0621BDF7D3FC314A1188201C0830BDF7CDFC10BD70B5FF230133C458002C03D0201CB5F710FF0CE0061CC518142099F763FF041E0ED02860321C25490023B5F7E3FE244A11682448BDF7CAFD011C201CB5F7E5FE71
:FB76700070BD10B5041E13D0F830006840070FD5201C28308DF74DF81B490B68FF2B01D08DF769F8E069F821884340210843E06110BD10B5041CFFF7E4FF13225C23195B002093F7C4FBE0690006C00E0A2803D10A21201C78F7FBFF201C7EF7D0FF201C7FF7FBF8201C7EF7E7FF206877F743FC10BDC04692AC0900E2AA0900F3450200E4AA0900D43000008C06080010B5AC4AAC4900780302AC4C20680004184308601078C3020868184308606068000423681B0C18434860507888600020C860012010BC08BC184710B5041C00290AD18DF769FD70342078042815D19C484379012B11D10EE0022906D15030407F76F793FC0023A38107E0052905D10078
:FB776B00F0E7F8002801D18DF72FFB10BC08BC184770B5904D2B68FF2B56D1002077F756FA2860FF2850D001238B4803608B4803708B4C0323E3748B480168201C6FF793F825232374022363743323A374201C7030042303700023437023632384824803685B006384242000230355E3818DF7E7FF286877F7E9FC7D4E30607368802003437360286877F768FC211C503103680B77C269C8680726B0433240104301225202104380221043C8600023CB750B6813430B6001238B7702234B776D496D488DF71EFB201C6EF7D2FF012070BC08BC184770B5061C041C0023674803605F480378002B04D140235C490B60980527E04B0704D570342078042867D1D4
:FB78660044E08B0724D5351C70352B78022B5FD16978564802685A4803684B43301C934213D95300638418360123737304232B703323A37400236B706FF738FA2023474E3360D80578F707FA42E0013169701EE0CB073DD5351C70352878022838D315D0042817D334D147490868430E47490B6047488DF7BAFA02232B704823A37440490B685B006384183401236373301C6FF70DFA1DE0102331480360180678F7DBF9334803685B00638418340123637304232B7000236B70301C6FF756F835493548062202F0F6FF002802D133486FF74CF870BC08BC184731498868002805D0007C2438012801D8012000E00020704700B51D211C4803F015F819212791
:FB7961004803F011F8FF23274A1360144A13600023264A1370FF23254A13608DF72AFA00BD10B583B0041C0C22E92109036846BCF7F8FF694600200A7801312254174B1A5401300628F7D34B78A37103B010BD25AE0900B8890E0038800E00A42C08008C060800D4500800BEC10800F0500800B00608009006080000820E00D85008006400080018800E009806080098830E00E4500800E0500800CAAD0900E8500800645108006C21080088060800BFC10800F4AA090000B5002346490B7046490B7046486FF713F846490868FF2804D077F79AFAFF2342490B6001234248036042480378012B04D18DF7F8FD00233E490B7000BD10B5041C70342378022B2C
:FB7A5C0024D13B4B1968043B1A68CB0717D4530315D54B0313D50723DB040B400FD153061A0F032A0BD18B05DA0E082A01D00C2A05D13048FFF777FF0323237006E0CB0704D46378013363706FF735F910BC08BC184730B582B0041C27490B7E002B39D126490B68702003401D09A37BAB4231D023490B68FE20034000D00123002B26D10020B2F74BFE002821D11E490B689B061DD48BF781FD002819D16946281C99F7E6FF68466FF76DFE68469AF713F800209AF773F81448002343628362009B9B089B00416B59180B011B09436302E0A07B9AF763F802B030BD5CC80800BEC10800F05008008C060800D4500800BFC108002C8B0E00F0AB09002C2D085E
:FB7B57000024860E00B4C4080008800E006C210800037B0C30FF2B04D14378202B01D1002000E001207047F0B582B00C1C01D10420A3E0051C52480268002A08D0281CC3F78BFE002803D0FF300006000E95E0F82148590007800F01282DD1E86900042AD4237B5B0827D047490868800723D5201CFFF7CEFF00281ED0281C28308DF7B3F8F822505902229043F8225051201C99F7ABFC0821281C7EF7FFFB8CF7E6FE0123394A1370394A1168281C8CF7CDFE281C8DF709F8BBE72F687B0135481E18F37F012B55D0237B5B080ED1637B052B02D1304900910DE030490091042B09D0DB002E48C218009204E0201C0C307AF7D0FC009000990B7963770023CC
:FB7C5200236002F088FE01900099486840010BD4B068002805D003682360B3681C60B46011E0B46024600EE0F068002805D003682360F3681C60F46001E0F4602460211C281C90F702F80123BB401649086818430860019802F067FEE8690006C00E0A2803D1381C73F71BFF09E0082807D1381C6CF7CEFD03E0201C99F739FC5AE7002002B0F0BDC046BCC80800641B0800BFC10800885008007C290800E8A90900F0A909006CCF05007429080070B582B0002301935F490868202800D1B6E010285AD15D49086877F7D5F9051C5B4E301C76F7F8FE002811D0041CF822135801221343F8221350EB69C06907210B4088431843E061286877F70EF90CE02CCF
:FB7D4D001C311C281C28300622BCF715FEF820435902208343F8204351311C201C8CF75BFD002805D0F820035901200343F8200351201CFFF756FC02F0F0FD012321688B40404A11681943116002F0EFFD20686CF76FFCE369F820834310200343E361206801216CF7D3FD201C8FF70FFE201CFEF7C6FEFF233148036059E0FF23013398424AD12E4876F79FFE041E50D077F70BFBE369012000068343F820834310200343E361E36C5B005B08E364EC210B59000683430B51201C00217BF783FB201C00217BF7DAFB6B4601AA211C4C31201C283096F7DAF9002806D0019B002B03D0201C7AF7D2FF03E0211C002077F7B4FFFF231248036014480368012B3A
:587E480018D1E3691B0415D411480368002B03D1104803680E4803608CF776FC0AE0402802D18DF74EFC05E001235B02984201D18DF7DFFB012002B070BDC046D45008008C060800E8500800B4C4080088C8080088500800ECAA0900AB
:087EB800FFF7F9FD6EF7E0FF92
:FB7ED0009F48002303608360704770B59D490B68180A9D4A402803D19C49D1609C4906E09C490143D160030219189B4BC9189B4D29609B4C9B4963685B0E2468E407E40F634009D0402807D17F2464020B68964D2B400125ED0406E0FD2424020B68924D2B400325AD040B600B682B430B6000238E4E336003040B21090459182143032631438B4E31600F30106070BD10B57C4A1368002B05D0612101220A546EF7D1FE05E0041C6EF72BFD201C00F0B0F810BC08BC184710B5041C7E48416A002902D1836A022B09D9032904D1836AFF203630834202D2201C6EF76DFF60237648195D405C80210143754A11606D480368744A136043681720800603435387
:357FCB0060FFF785FFA37B704A136000236F4A1360082113206DF7DDFD10BD30B5041C002927D1FFF7C9FF6A4D61342178694A0023D0560129B7
:FB80000007D17DF72BFF0006010C2868654A104006E07DF723FF0006000E2968090A0902084328604A4A11685F484143494A1068000A0430BDF7E2F85C4A106014E0022907D101235A490B604034607F76F71BF80AE0052908D1002355490B60FFF76EFC002801D18CF7B6FE30BC08BC184700B5374A011C1368002B0DD09368002B0AD19389936060310A780023022A00D2531C0B706EF73EFE08BC184700002C49037D022B07D10868431E00D30B608868431E00D38B60704710B5037D092B0CD13D4C3D4A106877F776F8206060688021884360603A4AD078206210BC08BC184770B583B00024364E4E256543AB19991C3548062202F011FC002803D00147
:FB80FB0034042CF1D305E0A919487800020978084300E0002001A9C8700821000A02AA1070012301A883706846831D2848032292F783FF03B070BDF0B5061C0F1C054C6368FF2B45D1012076F779FD6060FF283FD100207FE0F0AA090094060800C8890E0040C07DC0447E000000D07DC0043E00008C800E00F8AB0900B88A0E00FFFFC3FF94830E0098830E006C210800A8060800A4860E0040820E0000830E00F8800E0004830E0092030800FF00FFFF710200009C830E00F0FC0E0000820E00F4AA0900CAAD090092AC0900B7C10800B6FC00002A4D0123EB742169281C6EF77CFB2760A389A3602649794326480068000A0430BDF706F8244908602423B6
:AC81F6002B7402236B743123AB74281C6030002303700123437000238370C3702B625D2002234355606876F7CAFFA8730123EB73184F391C301C8CF71DFE606876F7BFFF391C6EF7C0F9311C13480622BCF79FFB2169281C6EF751FB0120F0BD09480368002B00D00123002B09D0007D002806D0072801D0002000E00120002800D0012070476451080071020000940608009C830E00F8AB0900CAAD090000B5F8210B585B0702D4042180F796FA00BD9D
:FB82AC0030B5051C041C08790002C9780843012176F78BFC002802D112232B700EE00834F42109584907490F00D00121A1715C300088E071000A20720323EB7030BD000070B582B0051C0024200123181B0145481E18F821885940071AD4306876F754FF6968884214D1301C77F77AF800280FD03D4B69460B8002238B705C23985BC870000A01A90870394A6946301C81F700F801340B2CD8D30123354A1376686872F7A8FD686873F7BCFA6868B2F7E9F8696830486EF79EFD69682F486EF79AFD69682E486EF796FD69682D486EF792FD6C68002C45D10C2363432A481D18A87A022831D304280ED32ED1281C82F77AFE061C288000236B72E87976F78E95
:9183A700FEA03006810C3028E0281C82F76CFE288000236B72EB7999005B189B011B495E18311CB831487100230B71C436B379002B15D073792B80B3796B8033796B72281C82F751FE7071301D07E0002807D0281C82F749FE2880281C09300023037001340E2CB9D302B070BD88380800530C000043720100CC2F0800B42E0800682E08001C2E0800D037080040490800140B0800C2
:FB849200F0B5051C13235B049F4F3B60082105206DF77CFB9D4F3B689D4803403B603B68C00703433B608B4F3B6802273B43894F3B60974C984820620123974F3B60974FB868606278686065A8692430C17880220A43934F3A60934E8378B07B002B0ED1924D0021B0F7A5F8B169081C243042781302007B18430022B0F7B2FA09E00121B0F797F88A4D8A4A13680120400603431360884805608848838A8848036000232360F0BD0523838183692633187801280FD10021CB4382490B6000234B607D490B68802003430B607A490B68800403430B60704700B5C369002B23D013235B04694A13605F4A13685D4A13605B4A1368594A1360554A1368644A133C
:C3858D00607248724A11684160724A11684161714A11688160714A13680360704A1368704A136061486EF785FA08BC1847000030B5052383816C4A116806220A40062A02D181692A3108E08B0702D481692C3103E04B0704D481692E310B8801330B8013235B0449490B605049CB69002B12D1524C2568C37B012B0CD12368802083432360022099F7BDFB80231D43A06899040843A060256030BC08BC184713235B043A4803604148C369002B02D1434803680360704700B5002901D1FFF724FF08BC18470000FE
:FB87C000F0B581B0051C0C1C08790002C978084352D00020ADF70EFBFF2801D109234CE0071CADF7C8FA0023038121790902E27811438186C186051C83F711F82E1CB03673885808E8806379252B0ED2394800900521BCF7D9FB6179C8084907490F01228A40009B195C11431954B07BFF233D334343314819180091281CAFF7C4FC2F4885662521281CFDF7DBFF307B0021AFF7F9FE0523AB80381CAFF744FD00999E3101200870381C002100F035F8A279E179381C00F005F801E012232B7001B0F0BDF0B50C1C171CADF776FA061C201DB4F755FB051E1ED0B18D0B051B0D012040031843210408432B1CA907890F01D1186006E01870000A5870000A98FE
:FB88BB0070000AD8703A06120E2104090C281D91F7D1F8281CB2F7C0FEF0BD30B50C1CFF233D3343430548C51802F040F8A2352C8002F044F830BDC046F44E0800349D080038B0080000B5C37B012B05D1A9490B78002B01D101230B70B2F7CFF908BC1847000000B52C22A449A448BCF72DF8A348A34B1860A3494160A3498161A349C16100BD30B5041CBE342178FF233D334B439F495918FF2208328B18FF2119709D493C30062201F0DAFF00280CD19A4D23782B6002236B717F21C943A81D072201F0D5FF00232B7130BD30B5041CBE342078FF233D3343438E495D18203082F7A8FB281C6EF755F885F777FB8B48036821788B4203D1FF23036000230E
:FB89B600437130BD00B5017D032901D0042902D1B2F7DAF909E0037D062B02D100F008F803E0092B01D1B2F700FA08BC1847000070B582B0051C041C8034E37A002B08D0036DBE3319780820AEF73FFC0023A376E3726378032B28D0A87B98F763FF4008218C431A1E04360C618C00291DD08E421BD36078012806D1688CBCF70CFC062803D13E2002E0042803D008202B6DAF33187003236370281C6DF7BEFF2B6DBE3319780520AEF711FC31E06068002808D00090002301936946A87B99F785F8002363606378032B11D0FF201930285A864209D8A87B85F7A5FA002804D1281CB2F7DFFC002802D04E49C8780CE06378002B07D14C4BA87B185C0328020E
:FB8AB100D24949887801E047494878A874281CB2F7BBFB02B070BD70B5041C0E1C384D2878002802D0013828702878012804D83F4A13683F490B401360002816D0201C9830C378002B02D18188CA060ED58379002B11D0311C201CB0F709F92B78012B0AD9311C201CB0F7D5F805E0201CAFF79AFD201CB2F743FB70BDF0B581B0041C051C80350027AF81EF76FF230533C618F37D0133F375C37B012B13D17378002B19D1254803689B0715D5A07B98F7BDFE80084100A06981420DD098F751FE4000686008E00123737017480378A3740123DB07B361B77018480068009083075DD516490B685B0602D40098430732D5A07B98F79BFE400828846B78012B03
:FB8BAC0020E0C046FDCC080078E4050038AC090078150800BB8909002B8B090001890900349D080009C1080030AB090074150800E3C008001C800E00FFBFFFFFBC8B0E004015080008D102236B70236D588900016884201CB2F7C0F9F37D012B07D17DF71FF9011C201CAEF7B6FB01F0EFF92C484379022B14D1236DBE330068197888420ED17DF70DF9264B991D1A7988541879411C0720BCF718FB214B1871214B1F707DF7FEF8B074009906220A40062A1ED1236DBE33187885F7EAF9201C00F0A6F8F078012804D8184980000B5C01330B54E37B0099201C002B02D1FFF71FFF01E000F054F8201CAFF7E0FCAF7214E0B7758B070AD5A87A0D490B789856
:898CA7004205D2E37B002B02D00130A87206E02B7E002B00D02F76201CB2F775FA01B0F0BC08BC184730AB090086030800ECB008001CCD0800F0B5061E20D00768002F1DD0407CADF744F8051C707C182141430C484418786890F7E3FC98F764FC381C98F71BFC00233360217A01312172217A05480278A88D90F718FC00232372F0BDC046F4B008007C150800F7
:FB8D380070B5051C0E1C041C8034A37F002B1ED0AFF7E9FF184A537C012B09D9E37E002B02D1A08BC10603D5311C281CAFF7AEFFCD23585D00280AD0FF230533E818837D002B04D04378002B01D1012383700B490B681B070FD56378022B0CD1FF201630285C002807D0A0898004800E0023002800D10123237670BDECCC0800E02C0800F0B5041C051C3A4806689835A8880712F306D90FE9707307D90F0307DA0F002F04D0344803685B0300D5111CFF231533E0184378002B03D1002901D0012343708A4216D0AB79002B15D1002F08D0D0231859C168C91BC16002D48368DB1983600122AA71201CB2F703FB201CAFF7F6FA01E0002383713307DA0FA8E9
:FB8E3300884307D90F8A4234D11C4F397C0A0702D5B304990E2DD1184A13689B0303D5B3079B0F032B25D004214840A880251C5035AE87B304980E1CD020221149BB68181D01F070FDCC342078800712D50D490B68012080030340580B0BD02B68BE331878ACF76FFFAF303D210170012028870023AB87F0BDA88B0E00E02C0800ECCC080080980E00BC8B0E0010B51F4C2068002805D08008800098F739FB0023236010BDF0B5051CC668B469002C16D0B0F7ADF8002812D1154F3A1C211C1331E01CAFF785FF381C00F00AF80023AB60EB60A008800098F71BFB0023B361F0BD00B582B0262369460B800190081C76F79FFE02B000BD00B54368002B04D0B2
:1A8F2E0010220448002192F77EF800BDC046E49C0800DBAD09001720000078
:9C8F6400F0B583B00291FF233D3343432248C618356D01F0F7FC371C90372C1CB0348E239A5B02998A1A1204120C638853433A6FD21851014909019101F0ECFCF37B012B0ED16B8B5B000093288B4000019A101841014909181CBCF73BF9A0800098E080281C82F72AFCF37B002B0ED1E68870086883A188019898F719FCE288011C101CBCF726F9301A400828830298431E3B800123BB7203B0F0BD349D080030
:F4900800F0B581B00090ACF7B2FE041C0027364E336BDB071FD5B4421DD0251C2C354223A97D9A5D914216D1291C1031301C3C30062201F06DFC00280DD101F091FC051CBE36307800F036F8281C01F091FC3078AFF768F903E0C03601370F2FD8DB0098B2F7B9FA251C0123EB852C35201C80F7A1FD00980021ADF7A1FF1C4A13681021DB0603D5A971201CB3F72DF9201CB1F7EBFABE342178FF223D325143144BC9187F23FF2023300B54A623FF2017300B5401B0F0BD10B5FF233D3343430C48C418201C80304178012907D1418C608CBCF7B9F8062803D13E2002E0042903D00820236DAF33187010BD2890080040150800349D0800B1
:BC910400F0B5061C046D2B4803689E4201D1B0F701F8301CAFF73DFE351C8035288901380ED32881288904236B70002808D1301C6DF74BFCBE3421780520AEF79FF838E0687800281FD1B07B98F7C5FB4008B034A16898F75BFB01239B0698420CD267883B1859014909381CBCF746F87843A168081840014009A060A06800236B700223F374B06112E0022810D1AB7E002B0DD0E889298A431A1804000C074B984205D2EB7A002B02D1301CB1F795FF301C6DF7AEFDF0BD6C210800FF7F0000C4
:8C91FC00F0B5051C1F49FF230533C418E378980000230B544318581C00230370AF692B6D1889421C267C688C5043B04063681B1858014009381A01239B06984220D2B31D20789840A368D901EB7B002B00D15143E268824200D3101CBBF7D2FF011C802800D980219F352970074803789E4202D2701C207404E000230434191C381C0BC4F0BDC046ECB008006F150800EF
:E4929400F0B5061C071C9C373888102101401D490BD01D4BF518EB7898000A5C9301AA68D218AA604318597811E0174BF518EB7898004118487800280DD08C78097861438901BBF791FFA9680918A960211C8B01E868C018E8602B7C002B11D1E86800280ED0AB68D901F37B002B03D1336D1A8901325143BBF778FF802800D98020F870F0BDC046ECB0080004010000F0B50D1C114C20600B68DB0701D598F76EFA0F4E0020706637680E483840306098F77AFD98F778FD2868E0606868A0600220706698F770FD98F76EFD98F76CFD37600020E060A060F0BDC04600820E001C800E00FFFFFFFD41
:3093800000B54068084A13681979002909D1074A13681B0605D4002801D098F7D1F8012000E0002000BDC046C04F0800E02C0800D8
:7893CC0030B5041C80304378002B1BD10323E374252101230B55837E002B07D0236DD98B09014184A36903840123C372618CA06974F788FC238C984204D02084216DB03188800880FF230133E158E518A06998F7F9F9216DB2310A88011C101CBBF7E8FE011C201CB1F73CFFA3692B60201CAFF74AFE00236B7130BDE1
:FB945400F0B581B02F4806682F4805682F480378002B52D12E480368AB4203D12D480368B3424AD02C4C2D4FFE20284007D1002D03D02B480368DB0301D5002E1CD063681B071B0F022B02D0022098F74FFD25480078606324480078A06366F7CDFE01F071FA822141432068642250436430BBF79BFE431C3B6018E063681B0702D0002098F734FD00206063A063184A13680093174A1088392109014143181CBBF784FE386014490098BBF77FFE134908603868A06107490D6007490E6001B0F0BC08BC1847C04614CD0800B4C4080008C30800B8CA080010AB09000C000F00DC5E0800FC0A080009C308000AC30800C02D0800E80A080020CF01009C000F68
:75954F0000381CFFF7F4F902B0B1F7FCF8FFF712FAB1F709F930B5041C13490B685D78B0F769FE022C01D0042C16D1281C203081F7B5FD042C07D10D4800231A1C191C91F751FD022102E0022C03D10821281CADF711FD281CACF78EFC05490B689879012801D1ACF7F0FC30BDC49C08000E200000C89C080048
:FB95D400F0B5041C00216DF758FF002803DA01234E4843716FE0061C251C7835687A00280DD1A07B98F76FF94008236DB833196898F70BF9002804DC687A002805D0002E03DD201CB1F7C9FD55E0E37B012B03D1002801D101236B72A878802101433C4A1160082105206CF7B0FA384A5379002B41D1AFF767FD374F381C052101F09AF903233B74201C00F037F8AFF718FDEB8A002B0AD1FF201630205C002805D1AFF751FD3B7C082003433B740023AB74FF230533E6180023F375201CB1F794FE264A13780021002B00D101211170F078FF2806D16B7A022B03D1081CF070A3697360012805D8F1708B001C48C0187B7C8370201CAEF7B9FEF0BD30B584E3
:6D96CF007C18490B788374051C012200216DF775FDAC742C6DB223195B0239884200DB081C11494143E5208000BBF780FDFF210531695C884200D3081C32342178490701D5012801D8002800D101200349487430BDA42C0800A4860E00ECCC08006C150800ECB008007415080071020000F1
:FB974400F0B583B0012100910027C0237B431A481C18206BC00729D5251CBC356B78002B24D1261CE38D2C36002B1FD0B379002B02D00021009119E0211C0C310F48052201F0C8F8002811D00223B371201CB2F736FD01A9201CB2F71EFD01A9A878B1F7B8FD082201A9A878B2F73AFE01370F2FCBD3009803B0F0BD28900800004F080010B5002912D140498B79002B0BD03F490B69834207D13E4C2368DB0603D54631012008700EE0AFF75DFE0BE0022909D1011C48318A880B7E9B18013383814B889B1A4B8010BC08BC184730B5314A11680B06D90F884218D12F4D2C68ACF7A4FBC1780B02817819430279130419434279130619438C4208D12A1F1333
:FB983F00681A0C41780B0200781843824201D0002000E0012030BDF0B583B0051C00910026041C58342379002B2CD0012601A8B0F72FF9071C6379002B13D0E378012B07D13023585DFFF7C3FF002801D1061C19E02835AB79012B04D101A9381CAFF7CDFF061C0F480378002B0CD0012F0AD1029B03208003034001208003834202D1012300980360301C03B0F0BDC046AC210800642C080008800E00A88B0E0088980E006C9C0800F0B50D1C041C002D14D14B488379002B0CD04A480369A34208D1494A1368DB0604D5031C46330120187036E0201CB0F7C1FC32E0FFF754FF022D2ED1414A131C5421085B0004271C52373988084318644433251C563591
:FB993A00A807800F01D12E6808E02D1AC0002968C1402026301A6E6886400E431E60A36B002B0CD1A06EC16B91603C30457908212D0200792843D06013680B431360A06E806A9064F0BC08BC1847F0B582B0041C051CAFF767FF58352B79002B31D0EB78012B10D1201C28308379012B0BD16B79002B08D1007AFFF72DFF002803D1201C6CF7A2FB1DE0EB78012B1AD8A66E6846B0F781F86B79002B0CD1071C6946301C3C300622BAF7D1FF423637706C340120207012E02E231B5D012B02D16946AFF71FFFA37C0B498878834202D1201CB0F774FD201C0121AFF71EFE02B0F0BC08BC1847AC210800642C080008800E00808B0E0074150800034B04480397
:479A350060044B044803607047C04660AA0900501508008CAA09006415080010B5041C6CF755FB201C6CF7B8FF4A23002018536523195D0220ADF709FCA36EBC3318780021AEF7E5FD10BDDB
:149AA40000B5011C32310B78FB2213400B70ADF7F1FF00BDBA
:4C9AC800F0B5061C0F1C104D2C68A07B97F701FF80084300991C608CA26983185801400997F792FE041C002F0BD0B17B2B68987B6DF7C7FE002804D1032C01D8002400E0033C201CF0BDC0466C21080003
:FB9B1C00F0B586B0061C4568039581780A07120F0092C07802908F0943191A79059200200490C04A13681879002804D1BE490B681B0600D4C9E10098062800D9CAE10598002808D0122806D0301CAEF78FF9002800D1BAE1BEE1B54C2378B5490879834202D3201CADF77EF9B1484188002923D00378002B10D06378002B04D0AD4898F769FA002818D000236370A370A84A508850214143A74805E02378A648002B04D15022514398F70BFA06E098F753FA002802D0201CADF756F920782923191C41430191E11C8807800F01D10A6808E0091AC0000B68C3402022101A4A6882401A430198954B0099C95C815480180099032901D0052957D18C4A13681BF1
:FB9C17000600D44EE1477002998B1F0372291C09300622BAF7ABFE0635E11C8807800F01D10A6808E0091AC0000B68C3402022101A4A6882401A43019880180230291C0622BAF794FE0098052817D10635E11C8807800F01D10B6808E0091AC0000A68C2402023181A4B68834013430199C8180F30029A0C3A291CBAF779FEE11C8807800F01D10B6808E0091AC0000A68C2402023181A4B68834013430199C8182830F17872688918C9780170FEE0FF07FF0F0098042806D05C4A1368F17870680818C078587259490868C379012B18D1391C281CADF7FCFB009A042A05D1ADF719FC002800D1E4E04CE0FF2803D1391C281CADF742FCADF722FC002800D17D
:FB9D1200D8E040E050490B78002B3CD0009A042A17D14D480490291C1030062200F0F3FD002800D0C6E00499887D03071B0FBB4200D0BFE08023034000D1BBE04006400E1FE00922835601200856834200DAB1E03E480490291C1030062200F0D4FD002806D10499887D03071B0FBB4200D1A1E0291C049810300622BAF7FBFD8023381C18430499887501210491E11C8807800F01D10A6808E0091AC0000B68C3402022101A4A6882401A43019880184770291C02300622BAF7DDFD20480378002B19D0E11C8807800F01D10A6808E0091AC0000B68C3402022101A4A6882401A4301998818F17872688918ADF7E3FC0006000EFF285FD106350298FA30003E
:EB9E0D0006000E02900098E11C012822D18807800F01D10B6808E0091AC0000A68C2402023181A4B68834013430199C8180021017225E0C04F0800E02C08005DC30800BC9C080093C3080014E3050068C30800B8AF08008807800F01D10B6808E0091AC0000A68C2402023181A4B68834013430199C818029A0272291C0930BAF77CFDE11C8807800F01D10B6808E0091AC0000A68C2402023181A4B68834013430199C8182830F17872688918C97801700498002802D023780133237023780A490879834202D3201CACF7D5FF0598122804D1AEF78DF8AEF7C2F804E00398002801D097F728FB06B0F0BDBC9C08003C
:FB9F0000F0B586B0041C012203920292002200923249051C08682035EB7A012B02D1304A117801E02E4A5178A17406220240062A51D12C4A16683207120F019201070BD529490B68987B002805D0301CAFF7FCFE0090029000E00390244F019805282BD1EB7A012B28D83306D90F287B414023D1ABF7FCFF79680491B968059104A90231062200F0C9FC002816D10398002813D00298002810D0201CAFF7C1FF009900290AD0201C6CF7ADF811490B68DB0703D4201C0021AFF76AFE0E490B681B060AD50198052801D0032805D1391C3004000C0022ADF700FA06B0F0BDC046BC8B0E005C150800A88B0E00B89C080080980E0008800E00E02C080010B556AB
:FB9FFB004C822099F731F9000600160022A15600290ED0CB10CA1AC310D2187F23DB439A4201DA181C04E07F207F2A01DC10060016010609162170494A1368002B01D14848C17710BD70B5002644480368002B01D184F790FC434C4449201C0F300522BAF793FC00252819C07B97F756FE36180135052DF7D33D48C36A5B011CD53C4803685B0518D400253B4803789E4213D001200A2D00D9022040194100374885F7E0FB002805D0291C201C0F3085F7EBFB013E0135252DE7D3211C0F313048052200F02DFC002809D0211C0F312C480522BAF75BFC63690120834363616369DB0707D4FFF732FB616901229143104001436161002070BC08BC184700B556
:96A0F60075F70FFA00280BD11F480368002B07D114490B681D490868834201D1012000E0002000BD00B5B821194800F032FC00230B4A137000BD10B5041C15480368002B0BD0201C002185F7A0FB1821201C85F79CFB4E21201C85F798FB10BDC0462CAE0900B4C4080050370800F4460800F44E08005420080020040800A4030800E0340800004F080010CD0800E4C708009034080014CD0800D5
:78A1AC0000B574F771FF002805D11848437D002B01D175F7B0FF00BD00B574F765FF002805D11248437D002B01D175F7A4FF00BD70B5051C0E1C0024C02363430C481818036BDB0703D5321C291CB1F749FF01340F2CF1D370BD00B5064875F780FF7CF7C9F813211620FFF7E3FF00BDE44E0800289008009C450800A2
:FBA31000002809D1104A1068104A1368984201D1012801D1002002E08800411AC81E70470B4A1068C306990F01290BD14007400F052801D8002801D1002001E002490868024908607047C046901C080064AC090004300E00002E02D00020E05504E0E35D002B01D0013BE3557BF7FBFB10B5A44C201C042100F000FB7F21C943A01D072200F0CAFAFF23236000239E4803709E4803709E4803709E4803709E4803709E4B9E4803600123DB029D48038080239D48037000239C4803709C4803709C480621BAF7FAFD14219B48BAF7F6FD14219A48BAF7F2FD10BD30B5041C98480368002B04D000230360282300201855944D00216962A96277F7D3FA92480357
:FBA40B0068002B07D174F740FE002807D18F48437D002B03D1012090F709FB04E075F76FFD2834042020700023894A137089480378012213430370FFF79BFF281C8A300621BAF7BCFD30BDF0B5061C051C081C08356C4C2368FF2B20D076490330062200F055FA002819D16079022807D12068ABF77CFCC38D012B10D1002711E001280FD1206874F719FEC1690906C90E0839062903D2FF210931475C02E0122333700EE0A11DE81D0722BAF767FA8021A01D072200F034FA00232371AF710823F370F0BD30B50C1C5B4D0331281C0622BAF754FA637A564803701422211C0A315648BAF74BFA1422211C1E315448BAF745FA002347480370434CFF23236087
:FBA50600281C0021ABF73DFC002803D1281C0121ABF737FC002806D0C38D012B12D1BE30007802210CE0281C74F7F1FA002809D0C2691206D20E083A062A03D2006801212060617130BD0B7935480370CB78304803707047F0B5052630480378002B50D12A4C2768FF2F4CD02079811D0720BAF77EFE05062D0E607902280CD1381CABF7F7FBC38D012B3CD1A31DEA560024012622490E7016E0012833D1381C74F78FFDC1690906C90E0B1C083B062B29D2A31DEA56FF230933C45C0123174803700A2900D10326144800211D4B1B579A420DDA0278013202700278B24212D301700F4A1378002B0DD091F795F80AE0154B1B5701709A4205DD0648037800CF
:FBA601002B01D091F76EF80120F0BC08BC184730AB090002C108000FC10800840308008603080010C10800C05D00009C070800A007080099070800D8C20800ADC9080009C1080011C1080025C1080024C9080054200800DCCC0800E44E0800EEC00800E00A0800381CFAF723FC6AF788F8281CFAF73CFC6AF7A1F881B000F003F873F7C2FA0000F0B5041C0D1C7BF7DFFB324E7379012B12D180213368095D8B420DD1A02210553179891988713079411C0720BAF7E0FD30710023284A1370271C261C6436317F9F2038569F377BF76EFB3870371CB37D0C37002B15D03368DB0508D41F4803691B010ED5301C8FF749FB002809D00023B3610123FB720023E2
:74A6FC00BB727B72301C8DF76EFB33685806000F295C002904D0144B185CB072431E0DE010490B69DB000BD5104A11680A6853031B0F984204D193025B0F013BA3810CE0012333723B68FF20013083433B600D2307490B70301C73F7EBFAF0BD30AB090086030800542008009EBB05001C2B0800E8C00800D5
:54A7980083780F2B02D1032311480360704700B50F480368002B05D0002303600F21181C79F770F900BD00B5094902060CD40868012807D102230B6018220F21002079F740F903E0032801D1022000E0002000BD0CAB090033
:18A80800044A1088012149020140480A012250407047C046E8C408002E
:FBA8800000B500F071F8002320490B7000F074F800BD00B51E4B984202D1081C00F001F800BD00B5012100F006F800BD00B5002100F001F800BD30B50C1C144D15490B78012B1AD10178032901D0082915D18378002B12D100F048F8002C03D02B7801332B7008E0041C2878013803D3287002208BF73BFF201C00F03FF830BD00B5FFF7D5FF00BD014908787047C0462DAE0900B8520800540008007847000000C09FE51CFF2FE1FC4005007847000000C09FE51CFF2FE1CC4805007847000000C09FE51CFF2FE1E05105007847000000C09FE51CFF2FE1741005007847000000C09FE51CFF2FE160E801007847000000C09FE51CFF2FE17CD7040078470061
:FBA97B000000C09FE51CFF2FE190D704007847000000C09FE51CFF2FE1304F05007847000000C09FE51CFF2FE1CC51050023000000494D090024000000454D0900250000004D4D090035000000594D090088000000994D09008D000000BD4D0900910000005BA509009200000000000000000000000300000259460200040001000000000000000000000000000000000000000000000000000000000095510200377709003D780900537A09000000000000000000000000006754020000000000B78009000000000000000000E77F09005D7F0900000000006F800900000000009D800900875102009F9504006D9904007F93040000000000C59709000000B1
:9AAA76000000A7960400000000000000000005990400C39304009F9504006D99040091A2040000000000E5980900000000008599090093A3040075680900A3680900C3930400420500005E04000062040000420500006C04000062190000440500006C040000621900000A00000001002100A08601000C0019000200000000180000FF000000800200008002000034AA090000180008030000000100000040
:E0BC000030B582B0041C30490B7E002B5AD12F490B68702003401D09A37BAB4252D02C490B68FE20034000D00123002B47D10020AEF7A2FD002842D126490B689B063ED487F7D8FC00283AD16946281C95F73DFF68466BF7C4FD684695F76AFF002095F7CAFF1D48002343628362009B9B089B00416B59180B011B0943631848016819E0251F237B212B15D1281C6DF7B5FC00984308606918184308990149096161E08BB9F7C8FAA083281C6DF704FB281C6DF771F807E00C1C09688442E1D102E0A07B95F799FF02B030BD2C2D080024860E00B4C4080008800E006C210800A80208001F
:00000001FF
